:100000000C942A000C9445000C9445000C94450077
:100010000C9445000C949A010C94C7010C94F901BE
:100020000C9445000C9438010C9445000C94450048
:100030000C9445000C944A080C941B030C94450046
:100040000C9445000C9445000C9445000C9445001C
:100050000C94450011241FBECFE5D4E0DEBFCDBF18
:1000600010E0A0E6B0E0EEEEFEE102C005900D92D9
:10007000AC3BB107D9F711E0ACEBB0E001C01D9289
:10008000AE34B107E1F70C94AD000C940000CF93AF
:10009000DF93CDB7DEB7E7E3F0E08FE18083E4E301
:1000A000F0E08EEF8083E1E3F0E084E08083E2E340
:1000B000F0E088E38083DF91CF910895CF93DF93C1
:1000C000CDB7DEB721970FB6F894DEBF0FBECDBF18
:1000D000F89480E29EE490934B0180934A01198248
:1000E0002FC08981482F552789819927880F991F0B
:1000F000FC01E252FF4F808191819C0128513C4FCD
:10010000CA01880F991FFC01E65CFE4F31832083F2
:1001100020914A0130914B0189819927880F991FBD
:10012000FC01E65CFE4F80819181A901481B590BBF
:10013000CA0190934B0180934A0189818F5F898323
:100140008981883070F2789421960FB6F894DEBFDA
:100150000FBECDBFDF91CF910895CF93DF93CDB781
:10016000DEB721970FB6F894DEBF0FBECDBF0E9459
:1001700047000E9416010E940D031092390188EB7E
:1001800092E09093D9008093D80086E093E090931A
:10019000DB008093DA0078948091C0008823E1F33B
:1001A0001092C0000E9405060E9444040E9471073C
:1001B00000C08091CA00813041F4809139018823C8
:1001C00011F40E945E001092CA008091C300813039
:1001D00021F41092C3000E94CB078091C1008130AE
:1001E00011F41092C1008091C000813011F410927E
:1001F000C0008091BF008130E1F61092BF000E94E4
:100200004C06D7CFCF93DF93CDB7DEB7F894E9E5AF
:10021000F0E089E180837894DF91CF910895CF93C6
:10022000DF93CDB7DEB7DF91CF910895CF93DF9302
:10023000CDB7DEB7E3E5F0E082E08083EFE4F0E005
:100240001082EEE4F0E082E08083EAE4F0E084EF04
:1002500091E091838083E8E4F0E080ED97E0918382
:100260008083E9E5F0E081E08083DF91CF9108951C
:100270001F920F920FB60F9211248F93CF93DF939B
:10028000CDB7DEB78091CF008F5F8093CF00809194
:10029000CF00833029F481E08093C3001092CF0017
:1002A000809138018F5F80933801809138018732C7
:1002B000C9F581E08093C100109238018091CE0091
:1002C0008F5F8093CE008091CE00853029F410920C
:1002D000CE0081E08093C2008091CC008F5F80933C
:1002E000CC008091CC00843641F41092CC0081E0A7
:1002F0008093BE0081E08093C0008091CC00823367
:1003000019F481E08093C0008091CD008F5F8093CD
:10031000CD008091CD008A3029F41092CD0081E08B
:100320008093BF00DF91CF918F910F900FBE0F9000
:100330001F9018951F920F920FB60F9211242F93B2
:100340003F934F935F936F937F938F939F93AF935D
:10035000BF93EF93FF93CF93DF93CDB7DEB7E091D9
:10036000D800F091D9000995DF91CF91FF91EF91DD
:10037000BF91AF919F918F917F916F915F914F91BD
:100380003F912F910F900FBE0F901F9018951F92C5
:100390000F920FB60F9211248F93AF93BF93EF93E9
:1003A000FF93CF93DF93CDB7DEB7A2E3B0E0E2E3F4
:1003B000F0E080818B7F8C93A5E3B0E0E5E3F0E093
:1003C00080818D7F8C9381E08093C9008091BC00F7
:1003D000883019F481E08093CA00DF91CF91FF91BA
:1003E000EF91BF91AF918F910F900FBE0F901F9023
:1003F00018951F920F920FB60F9211242F933F93CF
:100400008F939F93AF93BF93EF93FF93CF93DF931C
:10041000CDB7DEB72297DEBFCDBFA2E3B0E0E2E307
:10042000F0E0808184608C93ECE4F0E01182108233
:10043000A8E4B0E08091BC009927880F991FFC01C7
:10044000E65CFE4F8081918111969C938E93809102
:10045000BC00882339F4A5E3B0E0E5E3F0E0808157
:1004600082608C938091BC00282F33273A832983A4
:1004700089819A8182309105C1F129813A812330A5
:10048000310554F489819A81009789F029813A8154
:1004900021303105D9F04EC089819A818330910590
:1004A00099F129813A8124303105E9F143C0A8E36B
:1004B000B0E0E8E3F0E0808180618C93A8E3B0E0F5
:1004C000E8E3F0E0808181608C9334C0A8E3B0E081
:1004D000E8E3F0E080818E7F8C93A8E3B0E0E8E36E
:1004E000F0E0808182608C9325C0A8E3B0E0E8E36F
:1004F000F0E080818D7F8C93A8E3B0E0E8E3F0E04A
:10050000808184608C9316C0A8E3B0E0E8E3F0E05B
:1005100080818B7F8C93A8E3B0E0E8E3F0E08081FA
:1005200088608C9307C0A8E3B0E0E8E3F0E0808146
:10053000877F8C938091BC008F5F8093BC008091FB
:10054000BC00893010F01092BC002296F894DEBFF7
:10055000CDBFDF91CF91FF91EF91BF91AF919F916F
:100560008F913F912F910F900FBE0F901F90189574
:10057000CF93DF93CDB7DEB78091D0009091D100BB
:100580000097B1F4E6E4F0E0808191819093D70088
:100590008093D600AEE4B0E0EEE4F0E080818F7BA3
:1005A0008C9381E090E09093D1008093D0002BC099
:1005B000E6E4F0E0808191819093D5008093D400AF
:1005C000AEE4B0E0EEE4F0E0808180648C932091B2
:1005D000D4003091D5008091D6009091D700A90128
:1005E000481B590BCA019093D3008093D2001092FC
:1005F000D1001092D0008091D2009091D3009093BE
:100600004D0180934C01DF91CF910895CF93DF93FB
:10061000CDB7DEB7DF91CF910895CF93DF93CDB7FC
:10062000DEB7E7E2F0E01082E6E2F0E08FEE8083F2
:10063000DF91CF9108951F920F920FB60F92112460
:100640002F933F938F939F93EF93FF93CF93DF93DA
:10065000CDB7DEB7E6E2F0E010828091BD009927C9
:10066000E4E2F0E020813181880F991FFC01E25221
:10067000FF4F318320838091BD008F5F8093BD0049
:100680008091BD00873010F01092BD00E7E2F0E0ED
:100690008091BD008083E6E2F0E08FEE8083DF9101
:1006A000CF91FF91EF919F918F913F912F910F905B
:1006B0000FBE0F901F901895CF93DF93CDB7DEB785
:1006C000E9E2F0E080E18083E0E4F0E01082EAE239
:1006D000F0E088E18083E0E4F0E086E88083EBE20C
:1006E000F0E082EC8083DF91CF910895CF93DF9388
:1006F000CDB7DEB721970FB6F894DEBF0FBECDBFE2
:100700008983EBE2F0E080819927807290700097F6
:10071000C1F3ECE2F0E08981808321960FB6F89472
:10072000DEBF0FBECDBFDF91CF910895CF93DF9392
:10073000CDB7DEB726970FB6F894DEBF0FBECDBF9C
:100740009E838D838D819E81DC01FD0101900020BF
:10075000E9F73197CF018A1B9B0B9C838B831A820D
:1007600019820FC029813A818D819E81F901E80F9C
:10077000F91F80810E94760389819A8101969A836C
:10078000898329813A818B819C818217930750F755
:1007900026960FB6F894DEBF0FBECDBFDF91CF9186
:1007A0000895CF93DF93CDB7DEB780916A000E94A2
:1007B000760380916B000E947603DF91CF910895BC
:1007C000CF93DF93CDB7DEB766970FB6F894DEBF51
:1007D0000FBECDBF9E8B8D8B8D899E894AE050E0E8
:1007E0009E012F5F3F4FB9010E94FB0ECE01019683
:1007F0000E94960366960FB6F894DEBF0FBECDBF7B
:10080000DF91CF910895CF93DF93CDB7DEB72297D5
:100810000FB6F894DEBF0FBECDBF8A8387E0898311
:100820001FC08A81482F55278981282F332727FD0C
:10083000309581E090E0022E02C0880F991F0A9443
:10084000E2F7842395231816190624F481E30E9405
:10085000760303C080E30E947603898181508983F7
:1008600089818823F4F680916A000E947603809142
:100870006B000E94760322960FB6F894DEBF0FBE7F
:10088000CDBFDF91CF910895CF93DF93CDB7DEB782
:100890000E947D0463E080E00E94E1058CE690E028
:1008A0000E94830562E081E00E94E10587E790E015
:1008B0000E9483050E947304E0E3F0E080819927A1
:1008C000807290700097C1F70E947D04DF91CF91F4
:1008D0000895CF93DF93CDB7DEB78DE00E94B805C2
:1008E000DF91CF910895CF93DF93CDB7DEB78CE042
:1008F0000E94B805DF91CF910895CF93DF93CDB7D4
:10090000DEB781E00E94B805DF91CF910895CF93C3
:10091000DF93CDB7DEB726970FB6F894DEBF0FBED4
:10092000CDBF9E838D838AE090E09C838B831CC027
:1009300082E390E09A8389830EC08D819E81019726
:100940009E838D838D819E810097B9F789819A81DD
:1009500001979A83898389819A81009799F78B817E
:100960009C8101979C838B838B819C81009701F7ED
:1009700026960FB6F894DEBF0FBECDBFDF91CF91A4
:100980000895CF93DF93CDB7DEB721970FB6F894D4
:10099000DEBF0FBECDBF898389819927817090709A
:1009A000882341F0A5E3B0E0E5E3F0E080818061D9
:1009B0008C9307C0A5E3B0E0E5E3F0E080818F7E93
:1009C0008C938981992782709070009741F0A5E3FC
:1009D000B0E0E5E3F0E0808180628C9307C0A5E39E
:1009E000B0E0E5E3F0E080818F7D8C9389819927E9
:1009F00084709070009741F0A5E3B0E0E5E3F0E08B
:100A0000808180648C9307C0A5E3B0E0E5E3F0E06B
:100A100080818F7B8C938981992788709070009753
:100A200041F0A5E3B0E0E5E3F0E0808180688C93DD
:100A300008C0A5E3B0E0E5E3F0E090818FE789230B
:100A40008C9321960FB6F894DEBF0FBECDBFDF9119
:100A5000CF910895CF93DF93CDB7DEB7A5E3B0E094
:100A6000E5E3F0E0808184608C9381E090E00E9477
:100A70008704A5E3B0E0E5E3F0E080818B7F8C9311
:100A8000DF91CF910895CF93DF93CDB7DEB7229753
:100A90000FB6F894DEBF0FBECDBF8A838A818295E0
:100AA0008F70898389810E94C1040E942A058A81EE
:100AB0000E94C1040E942A0522960FB6F894DEBF58
:100AC0000FBECDBFDF91CF910895CF93DF93CDB708
:100AD000DEB721970FB6F894DEBF0FBECDBF898376
:100AE000A5E3B0E0E5E3F0E0808188608C93898144
:100AF0000E94430521960FB6F894DEBF0FBECDBF0E
:100B0000DF91CF910895CF93DF93CDB7DEB72497D0
:100B10000FB6F894DEBF0FBECDBF9C838B838B8155
:100B20009C81DC01FD0101900020E9F73197CF01A4
:100B30008A1B9B0B8A8319820EC0898199279C018D
:100B40008B819C81F901E80FF91F80810E94650566
:100B500089818F5F898399818A81981770F32496A0
:100B60000FB6F894DEBF0FBECDBFDF91CF910895D1
:100B7000CF93DF93CDB7DEB721970FB6F894DEBFE2
:100B80000FBECDBF898381E090E00E948704A5E37A
:100B9000B0E0E5E3F0E08081877F8C9389810E945B
:100BA0004305A5E3B0E0E5E3F0E0808188608C9345
:100BB00021960FB6F894DEBF0FBECDBFDF91CF9167
:100BC0000895CF93DF93CDB7DEB723970FB6F89490
:100BD000DEBF0FBECDBF8A836B838A81882319F461
:100BE0008B81805889838A81813019F48B8180546C
:100BF000898389810E94B80523960FB6F894DEBFD9
:100C00000FBECDBFDF91CF910895CF93DF93CDB7C6
:100C1000DEB781E090E00E948704A5E3B0E0E5E361
:100C2000F0E08081877F8C9383E00E94C1040E9462
:100C30002A0585E090E00E94870483E00E94C104B9
:100C40000E942A0581E090E00E94870483E00E94D0
:100C5000C1040E942A0582E00E94C1040E942A0564
:100C600081E090E00E94870488E20E94B8058EE04F
:100C70000E94B80581E00E94B80584E890E00E94D7
:100C800083056AE081E00E94E10589E890E00E9426
:100C90008305DF91CF910895CF93DF93CDB7DEB772
:100CA0002C970FB6F894DEBF0FBECDBF8091C40065
:100CB000882309F458C08091C700813009F051C0E1
:100CC0008091C400181634F48091C8008F5F80931F
:100CD000C80005C08091C80081508093C8008091F1
:100CE000C80088231CF483E08093C8008091C8006A
:100CF000843014F01092C8008091C800282F332748
:100D000027FD30953C872B878B859C85813091050D
:100D1000D1F02B853C85223031052CF48B859C85C8
:100D2000009761F01EC02B853C852230310581F093
:100D30008B859C858330910581F013C060E080E055
:100D40000E94E1050EC069E080E00E94E10509C053
:100D500060E081E00E94E10504C069E081E00E945A
:100D6000E1051092C400E0E3F0E0808180728D83A1
:100D70008D81882361F48091C700813041F4809196
:100D8000C800823011F40E94A90781E08D838D8113
:100D9000882351F48091C700843021F40E943308E5
:100DA0000E94710781E08D838091C700843009F033
:100DB0008FC0F8941C8217C08C81282F33278C8118
:100DC0009927880F991FFC01E252FF4F8081918182
:100DD0009695879596958795F901EA5FFE4F8083F2
:100DE0008C818F5F8C838C81863030F378941C8269
:100DF0006BC08C819927FC01EA5FFE4F80819927A7
:100E00009A838983CE01069629813A814AE050E08F
:100E1000BC01C9010E94FB0ECE010696DC01FD015A
:100E200001900020E9F73197CF018A1B9B0B8B8340
:100E30008C81843018F58C819927880F991F880F31
:100E4000991F682F80E00E94E1058EE890E00E94E3
:100E500083058C819927880F991F880F991F982FD8
:100E60008B81292F281B822F8D5F682F80E00E94A5
:100E7000E105CE0106960E94830523C08C81992747
:100E8000880F991F880F991F8051682F81E00E9459
:100E9000E1058EE890E00E9483058C819927880FF8
:100EA000991F880F991F982F8B81392F381B832FFB
:100EB0008D50682F81E00E94E105CE0106960E94C8
:100EC00083058C818F5F8C838C81863008F491CF71
:100ED0002C960FB6F894DEBF0FBECDBFDF91CF9139
:100EE0000895CF93DF93CDB7DEB781E08093C7003D
:100EF0001092C8000E9469040E947D0460E080E0B6
:100F00000E94E10581E990E00E94830569E080E0AC
:100F10000E94E10589E990E00E94830560E081E09C
:100F20000E94E10580EA90E00E94830569E081E08B
:100F30000E94E10588EA90E00E9483050E9469040E
:100F400060E080E00E94E1051092C400DF91CF9143
:100F50000895CF93DF93CDB7DEB784E08093C700C9
:100F60001092C8000E947D0469E081E00E94E105C2
:100F70008FEA90E00E9483050E94690469E081E0A5
:100F80000E94E1051092C4000E9473040E9416089A
:100F9000DF91CF910895CF93DF93CDB7DEB721973F
:100FA0000FB6F894DEBF0FBECDBF1982F894E0E310
:100FB000F0E08081992780719070009711F081E0B6
:100FC0008983E0E3F0E08081992788709070009732
:100FD00021F0898193E08927898378949981809190
:100FE0006900292F281B822F89838981992787FDF2
:100FF000909581709070882381F080916900982F7E
:101000008981890F809369008981982F92708091DE
:10101000C400890F81508093C40021960FB6F894C4
:10102000DEBF0FBECDBFDF91CF910895CF93DF9389
:10103000CDB7DEB7F894E0E4F0E01082E9E2F0E04A
:1010400081E08083E0E4F0E08EE88083EAE2F0E093
:1010500088E480837894ECE2F0E010821092CB0078
:10106000DF91CF910895CF93DF93CDB7DEB7F8949A
:10107000E0E4F0E01082E9E2F0E081E08083E0E487
:10108000F0E08EE88083EAE2F0E010827894DF916D
:10109000CF9108951F920F920FB60F9211242F93A4
:1010A0003F934F935F936F937F938F939F93AF93F0
:1010B000BF93EF93FF93CF93DF93CDB7DEB72C971A
:1010C000DEBFCDBF8091CB00282F332727FD309581
:1010D0003C872B878B859C8581309105C1F02B85C2
:1010E0003C852230310529F18B859C85009709F0DC
:1010F00080C0E0E4F0E01082E9E2F0E085E0808387
:10110000ECE2F0E0108281E08093CB0072C0E0E47A
:10111000F0E01082E9E2F0E081E08083ECE2F0E0D0
:10112000108282E08093CB001092F1001092F000C8
:1011300060C080E090E0A0E2B1E48A839B83AC834E
:10114000BD832BEA3AEA4AE250E46A817B818C81D2
:101150009D810E94C10ADC01CB018F839887A987FA
:10116000BA8720E030E040E85FE36F8178858985C9
:101170009A850E944B0C88230CF003C081E08E837B
:1011800018C020E030E04FE753E46F81788589850F
:101190009A850E94DF0B18160CF002C01E8209C04F
:1011A0006F81788589859A850E941009DC01CB01C1
:1011B0008E838E81898389818A95F1F78983ACE258
:1011C000B0E02091F0003091F100F901EA5FFE4FAC
:1011D00080818C93C90101969093F1008093F00077
:1011E0008091F0009091F1008233910511F41092FA
:1011F000CB002C96F894DEBFCDBFDF91CF91FF914D
:10120000EF91BF91AF919F918F917F916F915F917E
:101210004F913F912F910F900FBE0F901F901895F7
:10122000EF92FF920F931F937B018C0120E030E03F
:1012300040E05FE40E94150C88237CF020E030E061
:1012400040E05FE4C801B7010E94630A0E94810C7C
:10125000605070408040904804C0C801B7010E94AF
:10126000810C1F910F91FF90EF900895A0E0B0E0E6
:10127000ECE3F9E00C94300FFC016A0190819230AC
:1012800008F41BC1DB018C91823080F0943061F452
:10129000843009F012C19181EB018981981709F41A
:1012A0000CC1E4EBF0E009C1843011F4FB0105C18D
:1012B000823091F4923009F000C1EA01DF0188E048
:1012C0000D9009928150E1F78181FB019181892381
:1012D000E6018983F601F1C0923041F362807380A8
:1012E000EB018A809B80E480F580068117812C8148
:1012F0003D814E815F815301A818B908C501B7FC33
:10130000ABC080970CF457C0861497040CF4BEC091
:101310003401EE24FF2487019181FB01818198171C
:1013200009F4A6C0992309F49CC02E193F09400B6B
:10133000510B57FDB0C0E60119827B826A82F6012B
:101340002483358346835783E6012C813D814E817A
:101350005F8179018A01DA01C9010197A109B10907
:101360008F5F9F4FAF4FBF43F8F4E6016A817B81E7
:10137000A8019701220F331F441F551F6150704071
:1013800079018A01DA01C9010197A109B1098F5FC9
:101390009F4FAF4FBF4360F3E6017B836A83F60143
:1013A000248335834683578383E0D6018C9357FD8E
:1013B00039C0F60182C086149704B4F4C0E0D0E0CE
:1013C000DA01C90181709070A070B0705695479590
:1013D00037952795282B392B4A2B5B2B2196AC165A
:1013E000BD0671F78A0C9B1C681479040CF094CF2D
:1013F000C0E0D0E05401A618B708D801C701817039
:101400009070A070B07016950795F794E794E82A4D
:10141000F92A0A2B1B2B2196AC16BD0671F76A0C14
:101420007B1C7ACFDA01C901B695A7959795879568
:101430002170307040705070282B392B4A2B5B2B59
:10144000E6012C833D834E835F838A819B810196D5
:101450009B838A83F60131C0882799278A199B09C3
:1014600050CFE21AF30A040B150BA801970161CFC4
:10147000E60199837B826A822E0D3F1D401F511F1A
:10148000F60124833583468357838ECF20E030E0F6
:1014900040E050E041CF81E0E60189837B826A82AF
:1014A00050954095309521953F4F4F4F5F4FF60136
:1014B000248335834683578347CFCF01EEE0CDB7F2
:1014C000DEB70C944C0FA0E2B0E0E9E6FAE00C9431
:1014D000380F69837A838B839C832D833E834F836C
:1014E000588789E1E82EF12CEC0EFD1EB701CE01E4
:1014F00001960E94F30D8E010F5E1F4FB801CE01C1
:1015000005960E94F30D8A8991E089278A8BAE01A6
:10151000475F5F4FB801C7010E9436090E94D10C96
:10152000E6E0A0960C94540FA0E2B0E0EAE9FAE0FD
:101530000C94380F69837A838B839C832D833E833D
:101540004F83588799E1E92EF12CEC0EFD1EB7016F
:10155000CE0101960E94F30D8E010F5E1F4FB80160
:10156000CE0105960E94F30DAE01475F5F4FB801B3
:10157000C7010E9436090E94D10CE6E0A0960C94A7
:10158000540FA0E2B0E0E7ECFAE00C942C0F698372
:101590007A838B839C832D833E834F8358878E0170
:1015A000075E1F4FB801CE0101960E94F30DF1E1D5
:1015B000EF2EF12CEC0EFD1EB701CE0105960E9418
:1015C000F30D898D823078F09989923040F420E0D3
:1015D0009A8D8A89981321E02A8BB701E9C084305B
:1015E00051F4923061F020E09A8D8A89981321E0BD
:1015F0002A8FB801DDC0943029F4823041F764EBC2
:1016000070E0D6C0823079F3923009F32D8D3E8D93
:101610004F8D58A18D899E89AF89B88D222433249E
:101620002101AA24BB246501EE24FF24870160E088
:1016300070E00DC06F5F7F4F6032710599F1880FC8
:10164000991FAA1FBB1F569547953795279520FFD1
:1016500019C0280E391E4A1E5B1E662477244301DA
:10166000281639064A065B0628F4E1E06E2E712C36
:10167000812C912CAE0CBF1CC01ED11EA60CB71C19
:10168000C81CD91CEE0CFF1C001F111FB7FFD2CFC6
:10169000E1E06E2E712C812C912CE628F728082988
:1016A0001929C8CF8B8D9C8D2B893C89820F931F64
:1016B00002969C878B871A869A8D8A89981711F0D3
:1016C00081E08A87D7FE17C08B859C85A0FE0CC061
:1016D000569447943794279420E030E040E050E857
:1016E000222A332A442A552AD694C794B794A79419
:1016F00001969C878B8730E0A31630E0B30630E07C
:10170000C30630E4D30618F58B859C850EC0220CE9
:10171000331C441C551C019720E0A21620E0B206A1
:1017200020E0C20620E4D20680F4AA0CBB1CCC1C2C
:10173000DD1C57FEECCF31E0632E712C812C912CF7
:10174000A628B728C828D928E2CF9C878B87D6013E
:10175000C5018F779070A070B07080349105A1059D
:10176000B10551F0AD86BE86CF86D88A83E08987E1
:10177000BE01675F7F4F1CC0A7FCF4CF211431046A
:101780004104510479F380E490E0A0E0B0E0A80EB9
:10179000B91ECA1EDB1E80E8682E8FEF782E8FEFF1
:1017A000882E8FEF982EA620B720C820D920DACF18
:1017B000CB010E94D10CE2E1A0960C94480FA8E165
:1017C000B0E0E5EEFBE00C94380F69837A838B83FD
:1017D0009C832D833E834F83588781E1E82EF12C33
:1017E000EC0EFD1EB701CE0101960E94F30D8E0195
:1017F000075F1F4FB801CE0105960E94F30D89893E
:10180000823018F42FEF3FEF0BC089858230D0F380
:10181000B801C7010E94920E282F332727FD30956B
:10182000C901E6E068960C94540FA8E1B0E0EBE142
:10183000FCE00C94380F69837A838B839C832D831F
:101840003E834F83588781E1E82EF12CEC0EFD1E7C
:10185000B701CE0101960E94F30D8E01075F1F4F65
:10186000B801CE0105960E94F30D8989823018F4E3
:101870002FEF3FEF0BC089858230D0F3B801C7014D
:101880000E94920E282F332727FD3095C901E6E0EC
:1018900068960C94540FA8E1B0E0E1E5FCE00C94EC
:1018A000380F69837A838B839C832D833E834F8398
:1018B000588781E1E82EF12CEC0EFD1EB701CE0118
:1018C00001960E94F30D8E01075F1F4FB801CE01F4
:1018D00005960E94F30D8989823018F0898582303F
:1018E00018F421E030E008C0B801C7010E94920E50
:1018F000282F332727FD3095C901E6E068960C9420
:10190000540FACE0B0E0E7E8FCE00C943C0F6983D6
:101910007A838B839C83BE016B5F7F4FCE010196E0
:101920000E94F30D8D81823061F0823050F084305E
:1019300069F48E81882359F52FEF3FEF4FEF5FE772
:101940002AC020E030E040E050E025C02F813885FB
:1019500037FDF7CF2F31310564F78EE190E0821B20
:10196000930B29853A854B855C8504C05695479530
:10197000379527958A95D2F78E81882361F0509507
:101980004095309521953F4F4F4F5F4F04C020E069
:1019900030E040E050E8CA01B901E2E02C960C9436
:1019A000580F4F925F926F927F928F929F92AF9259
:1019B000BF92DF92EF92FF920F931F9320E030E0EF
:1019C00040E050E0FC01E480F58006811781D18081
:1019D0008081823038F4D801C701A061AF77B07040
:1019E0006FEFD9C0843009F46EC0823009F471C041
:1019F000E114F1040105110509F46BC082819381A2
:101A00006FEF823896070CF06AC062E87FEF681BC0
:101A1000790B6A3171050CF080C047015801062E20
:101A200004C0B694A794979487940A94D2F7442458
:101A30005524320181E090E0A0E0B0E004C0880FBE
:101A4000991FAA1FBB1F6A95D2F70197A109B10977
:101A5000E822F9220A231B23E114F10401051105F0
:101A600029F061E0462E512C612C712C8501740106
:101A7000E428F52806291729D801C7018F77907027
:101A8000A070B07080349105A105B10509F457C06C
:101A9000D801C701CF96A11DB11D60E070E0803074
:101AA000E0E09E07E0E0AE07E0E4BE0710F061E092
:101AB00070E027E0B695A795979587952A95D1F779
:101AC000AF77B07068C080E090E0A0E0B0E06FEF6A
:101AD00062C080E090E0A0E0B0E060E05CC08038F0
:101AE00091058CF7BC0161587F4FD801C7018F77F2
:101AF0009070A070B07080349105A105B105A1F07F
:101B00008FE390E0A0E0B0E0E80EF91E0A1F1B1F73
:101B100017FD28C0D801C701CCCF60E070E080E09D
:101B200090E0A0E0B0E0CCCFE7FEF2CF80E490E020
:101B3000A0E0B0E0E80EF91E0A1F1B1FE9CFE7FC8A
:101B400018C080E090E060E0E61660E0F60660E035
:101B5000060760E4160710F081E090E0BC01D801B0
:101B6000C701A7CF16950795F794E7946F5F7F4F4E
:101B7000D1CFD801C701805C9F4FAF4FBF4F60E00E
:101B800070E08030E0E09E07E0E0AE07E0E4BE07F2
:101B900008F48FCF8CCF282F392F9A2F9F77842F3F
:101BA0008078892B962F9795992797958F77482F2F
:101BB000492B6695852F8078862BD794DD24D79482
:101BC0008F77582F5D29CA01B9011F910F91FF909E
:101BD000EF90DF90BF90AF909F908F907F906F902D
:101BE0005F904F900895FC01DB012081318192814B
:101BF000492F4F7750E0991F9927991F8381682FAC
:101C0000660F692B881F8827881FFD018183662343
:101C100009F049C0211531054105510509F470C08D
:101C200082E89FEFFD0193838283220F331F441FBD
:101C3000551F220F331F441F551F220F331F441FF0
:101C4000551F220F331F441F551F220F331F441FE0
:101C5000551F220F331F441F551F220F331F441FD0
:101C6000551F83E08C932030F0E03F07F0E04F07F2
:101C7000F0E45F0790F482E89FEF220F331F441FC8
:101C8000551F0197203060E0360760E0460760E4AA
:101C9000560798F3FD0193838283FD0124833583E6
:101CA0004683578308956F3F71F1862F99278F5789
:101CB0009040FD019383828383E08C93220F331F36
:101CC000441F551F220F331F441F551F220F331F60
:101CD000441F551F220F331F441F551F220F331F50
:101CE000441F551F220F331F441F551F220F331F40
:101CF000441F551F506424833583468357830895BA
:101D000082E08C930895211531054105510519F4A0
:101D100084E08C93089544FD02C01C92BECF81E004
:101D20008C93BBCFEF92FF920F931F93CF93DF93D0
:101D3000FC01DB018081823050F09C91923038F0C0
:101D4000843041F49430B1F08181882381F461E0E2
:101D500070E04BC09430E9F18230A1F09230A1F3F1
:101D60006181ED018981681791F0662381F36FEF3E
:101D70007FEF3BC0EB018981682F77278181681B4A
:101D8000710933C0923059F560E070E02EC02281B5
:101D90003381ED018A819B818217930734F32817E1
:101DA00039079CF0E480F58006811781FD012481CC
:101DB0003581468157812E153F0540075107A8F20E
:101DC000E216F30604071507F8F6662309F0BFCFFD
:101DD000CECFFB018181882309F0B9CFC8CFEB01B9
:101DE0008981882309F0B3CFC2CFCB01E6E0CDB71C
:101DF000DEB70C94540FFB019F01E8944230C4F00D
:101E00004532B4F44A3029F497FB1EF4909581953D
:101E10009F4F642F77270E94630F805D8A330CF0F9
:101E2000895D8193CB010097A1F716F45DE2519390
:101E30001082C9010C941C0FDC01FC0101900020F0
:101E4000E9F73297AE17BF0730F47C916081708359
:101E500031976D93F7CF08952F923F924F925F92F3
:101E60006F927F928F929F92AF92BF92CF92DF92AA
:101E7000EF92FF920F931F93CF93DF93CDB7DEB70F
:101E8000CA1BDB0B0FB6F894DEBF0FBECDBF0994A3
:101E90002A88398848885F846E847D848C849B84FA
:101EA000AA84B984C884DF80EE80FD800C811B8108
:101EB000AA81B981CE0FD11D0FB6F894DEBF0FBE37
:101EC000CDBFED010895AA1BBB1B51E107C0AA1F9E
:101ED000BB1FA617B70710F0A61BB70B881F991FCB
:0E1EE0005A95A9F780959095BC01CD01089503
:101EEE004B2000000000003D00010D0A4550492D19
:101EFE005465737465720056657273696F6E203027
:101F0E002E3264006875687500416B6B7500202079
:101F1E000050504D2D4F75740050504D2D496E0090
:101F2E00444D582D4F757400444D582D496E004543
:0C1F3E0078697400000000000000000042
:00000001FF
